:020000040000FA
:0400000071303A28F9
:08000800A000030EA100831209
:1000100081018B100B11210E8300A00E200E090010
:0C007400203084008001840A6030040207
:10008000031C3C281230B0004B218316FF23900044
:10009000831283160C308505870183128501870141
:1000A000073099000030831691009F008312C830FA
:1000B00083168100831231309000003083168C004B
:1000C000831210308B00831600309B001C141A081A
:1000D0008312BC00831610309B001C141A08831274
:1000E000BD0083162F309B001C141A088312C30016
:1000F0006421831620309B001C141A088312C2004E
:100100000130C2080319C20081018E018F010B1159
:100110008B100B108C018B17A0203119A2202F21DE
:10012000B30B9E28031085190314B90DF030390262
:1001300003196D210F3039020319692171218C28AF
:1001400064000800080031110130B7008B13203023
:10015000370783169B001C141A088312A400103062
:10016000370783169B001C141A088312A300003063
:10017000370783169B001C141A088312A2008B17E2
:10018000321CC82822090339A200A309A409A50921
:1001900001303702031DD1283D18D1283D143E14EB
:1001A0005E2101303702031DDA283D1CDA283D109C
:1001B0003E146221DB28B70A023037020318080018
:1001C000A6280130B600B300B400B500B700850121
:1001D0008701B113A020B30B07290310851903145D
:1001E000B90DF030390203192529B41F8501B41F58
:1001F0008701B40B07293708B6080319B60003199D
:100200000529FF3085008700B6039630B400311D04
:10021000EA283111321C11292D090339AD00AE092C
:10022000AF098B1320303707BB002F08BA003821E5
:1002300010303707BB002E08BA00382100303707CE
:10024000BB002D08BA0038218B1785018701B70A3A
:10025000B60102303702031CEA28642108003E1C64
:1002600008003E101030BB003D08BA0038210800DD
:100270008B133A0883161C159A003B089B005530D7
:100280009D00AA309D009C1464009C1844291C11F8
:1002900083128B170800FF30D4000230D5000C30D9
:1002A000D600BA30D7003730D800DA30D9006F30F6
:1002B000DA00B830DB000230C10008000130BD00B8
:1002C000DD140800DD100800BD013D143D18DD14EB
:1002D00008003D143E145E2108003D103E146221CA
:1002E00008005C180516DC1885165C190514DC1965
:1002F00085145C1A8714DC1A07155C1B0714DC1BB9
:1003000087165D180716DD1887155C1C0512DC1CA6
:1003100085125C1D0510DC1D85105C1E8710DC1E1F
:1003200007115C1F0710DC1F87125D1C0712DD1C04
:1003300087118F08031908008F01C10B08004208BC
:10034000C1005408DE00EA22D4005508DE00EA228B
:10035000D5005608DE00541CEA22D6005708DE00FD
:10036000D41CEA22D7005808DE00541DEA22D80027
:100370005908DE00D41DEA22D9005A08DE00541EB6
:10038000EA22DA005B08DE00D41EEA22DB005C0809
:10039000C6005D08C700CA0BE3295408CA008B13C6
:1003A000831640309B001C141A0883125405031D49
:1003B0005C14831650309B001C141A0883125405D9
:1003C000031D5C108B17CB0BFB295508CB008B133F
:1003D000831641309B001C141A0883125505031D17
:1003E000DC14831651309B001C141A088312550527
:1003F000031DDC108B17CC0B132A5608CC008B1373
:10040000831642309B001C141A0883125605031DE4
:100410005C15831652309B001C141A088312560573
:10042000031D5C118B17CD0B2B2A5708CD008B13A6
:10043000831643309B001C141A0883125705031DB2
:10044000DC15831653309B001C141A0883125705C1
:10045000031DDC118B17CE0B432A5808CE008B13DB
:10046000831644309B001C141A0883125805031D80
:100470005C16831654309B001C141A08831258050E
:10048000031D5C128B17CF0B5B2A5908CF008B130F
:10049000831645309B001C141A0883125905031D4E
:1004A000DC16831655309B001C141A08831259055C
:1004B000031DDC128B17D00B732A5A08D0008B1344
:1004C000831646309B001C141A0883125A05031D1C
:1004D0005C17831656309B001C141A0883125A05A9
:1004E000031D5C138B17D10B8B2A5B08D1008B1378
:1004F000831647309B001C141A0883125B05031DEA
:10050000DC17831657309B001C141A0883125B05F6
:10051000031DDC138B17D20BA32A5608D2008B13B2
:10052000831648309B001C141A0883125505031DBE
:100530005D14831658309B001C141A08831257054B
:10054000031D5D108B17C4015C18C40ADC18C40AB3
:100550005C19C40ADC19C40A5C1AC40ADC1AC40A8D
:100560005C1BC40ADC1BC40A5D18C40AC50146181A
:10057000C50AC618C50A4619C50AC619C50A461AC3
:10058000C50AC61AC50A461BC50AC61BC50A4718AE
:10059000C50A3D1CE12A430845020318D82A45082C
:1005A0004402031808004608DC004708DD00080084
:1005B00043084402031808004608DC004708DD0031
:1005C000080044084502031808004608DC004708F4
:1005D000DD000800C001DE080319DE035E184014C8
:1005E000DE1A40144008C0015E1C4014DE1E401498
:0805F000C005C00C5E0C080000
:084000000E000300040008009B
:02400E00CC01E3
:10420000FF00FF00FF00FF00FF00FF00FF00FF00B6
:10421000FF00FF00FF00FF00FF00FF00FF00FF00A6
:104220000100FF00FF00FF00FF00FF00FF00FF0094
:10423000FF00FF00FF00FF00FF00FF00FF00FF0086
:104240001000FF00FF00FF00FF00FF00FF00FF0065
:10425000FF00FF00FF00FF00FF00FF00FF00050060
:10426000FF00FF00FF00FF00FF00FF00FF00FF0056
:10427000FF00FF00FF00FF00FF00FF00FF00FF0046
:104280000800800002000800040010000400200064
:1042900004000200FF00FF00FF00FF00FF00FF001E
:1042A00001000100010004000800040010000400E7
:1042B00080000400FF00FF00FF00FF00FF00FF0080
:1042C000FF00FF00FF00FF00FF00FF00FF00FF00F6
:1042D000FF00FF00FF00FF00FF00FF00FF00FF00E6
:1042E000FF00FF00FF00FF00FF00FF00FF00FF00D6
:1042F000FF00FF00FF00FF00FF00FF00FF000000C5
:00000001FF
